:020000040000FA
:020000000528D1
:080008008528850164008316C0
:1000100001308C001F3085001430950000308100C5
:1000200013309F0083120130900040308B0000306D
:100030009A000030C9001430CA005F200030C400AC
:10004000C30143140030CB006F204C08C7004D089B
:10005000C8004708C5004808C600FE30CF0016306B
:10006000CE004E088E004F088F000C108B17431CDB
:100070003A283728C30143144708C5004808C6007A
:100080000310C50CC60CFC30CF002230CE004E0849
:100090008E004F088F000C108B17431C50284D28E2
:1000A0008B13051E8516051A851258208B13B3284D
:1000B0000130CB006F204C08C9004D08CA00C301B5
:1000C000C314D830CF00FC30CE004E088E004F084D
:1000D0008F000C108B17C31C6E286B2808000310B0
:1000E000CB0D4B0D81389F000330C20081209F143F
:1000F0009F1878281E08CC0083161E088312CD0096
:1001000008008228C20B81280800C000030E831259
:10011000C1004E088E004F088F000C104318922823
:10012000C318A8280130C406441897289A2800004C
:1001300085169C2885129C2800000130C602031CED
:10014000C502031CC301410E8300C00E400E09000E
:100150000130CA02031CC902031CC301410E830003
:10016000C00E400E0900051E8516051A8512051ED3
:100170008516051A8512051E8516051A8512051E97
:100180008516051A8512051E8516051A8512051E87
:100190008516051A8512051E8516051A8512051E77
:1001A0008516051A8512051E8516051A8512051E67
:1001B0008516051A8512051E8516051A8512051E57
:1001C0008516051A8512051E8516051A8512051E47
:1001D0008516051A8512051E8516051A8512051E37
:0C01E0008516051A85120519B328192888
:02400E00E43F8D
:00000001FF
